 j2gss

 Timestamp is 1b576eee (reproducible build file hash)

 Preferred load address is 0000000180000000

 Start         Length     Name                   Class
 0001:00000000 00005850H .text$mn                CODE
 0001:00005850 00000036H .text$mn$00             CODE
 0001:00005886 00000092H .text$x                 CODE
 0002:00000000 00000160H .idata$5                DATA
 0002:00000160 00000038H .00cfg                  DATA
 0002:00000198 00000008H .CRT$XCA                DATA
 0002:000001a0 00000008H .CRT$XCZ                DATA
 0002:000001a8 00000008H .CRT$XIA                DATA
 0002:000001b0 00000008H .CRT$XIZ                DATA
 0002:000001b8 00000008H .CRT$XPA                DATA
 0002:000001c0 00000008H .CRT$XPZ                DATA
 0002:000001c8 00000008H .CRT$XTA                DATA
 0002:000001d0 00000010H .CRT$XTZ                DATA
 0002:000001d8 00000000H .gehcont$y              DATA
 0002:000001d8 00000000H .gfids$y                DATA
 0002:000001e0 00002120H .rdata                  DATA
 0002:00002300 00000000H .rdata$CastGuardVftablesA DATA
 0002:00002300 00000000H .rdata$CastGuardVftablesC DATA
 0002:00002300 0000006cH .rdata$voltmd           DATA
 0002:0000236c 000002bcH .rdata$zzzdbg           DATA
 0002:00002628 00000008H .rtc$IAA                DATA
 0002:00002630 00000008H .rtc$IZZ                DATA
 0002:00002638 00000008H .rtc$TAA                DATA
 0002:00002640 00000008H .rtc$TZZ                DATA
 0002:00002648 00000418H .xdata                  DATA
 0002:00002a60 000007a8H .edata                  DATA
 0002:00003208 00000064H .idata$2                DATA
 0002:0000326c 00000014H .idata$3                DATA
 0002:00003280 00000160H .idata$4                DATA
 0002:000033e0 00000388H .idata$6                DATA
 0003:00000000 00000080H .data                   DATA
 0003:00000080 00000838H .bss                    DATA
 0004:00000000 00000420H .pdata                  DATA
 0005:00000000 00000060H .rsrc$01                DATA
 0005:00000060 00000320H .rsrc$02                DATA

  Address         Publics by Value              Rva+Base               Lib:Object

 0000:00000000       __AbsoluteZero             0000000000000000     <absolute>
 0000:00000000       ___safe_se_handler_count   0000000000000000     <absolute>
 0000:00000000       ___safe_se_handler_table   0000000000000000     <absolute>
 0000:00000000       __arm64x_extra_rfe_table   0000000000000000     <absolute>
 0000:00000000       __arm64x_extra_rfe_table_size 0000000000000000     <absolute>
 0000:00000000       __arm64x_native_entrypoint 0000000000000000     <absolute>
 0000:00000000       __arm64x_redirection_metadata 0000000000000000     <absolute>
 0000:00000000       __arm64x_redirection_metadata_count 0000000000000000     <absolute>
 0000:00000000       __dynamic_value_reloc_table 0000000000000000     <absolute>
 0000:00000000       __enclave_config           0000000000000000     <absolute>
 0000:00000000       __guard_check_icall_a64n_fptr 0000000000000000     <absolute>
 0000:00000000       __guard_eh_cont_count      0000000000000000     <absolute>
 0000:00000000       __guard_eh_cont_table      0000000000000000     <absolute>
 0000:00000000       __guard_fids_count         0000000000000000     <absolute>
 0000:00000000       __guard_fids_table         0000000000000000     <absolute>
 0000:00000000       __guard_iat_count          0000000000000000     <absolute>
 0000:00000000       __guard_iat_table          0000000000000000     <absolute>
 0000:00000000       __guard_longjmp_count      0000000000000000     <absolute>
 0000:00000000       __guard_longjmp_table      0000000000000000     <absolute>
 0000:00000000       __hybrid_auxiliary_delayload_iat 0000000000000000     <absolute>
 0000:00000000       __hybrid_auxiliary_delayload_iat_copy 0000000000000000     <absolute>
 0000:00000000       __hybrid_auxiliary_iat     0000000000000000     <absolute>
 0000:00000000       __hybrid_auxiliary_iat_copy 0000000000000000     <absolute>
 0000:00000000       __hybrid_code_map          0000000000000000     <absolute>
 0000:00000000       __hybrid_code_map_count    0000000000000000     <absolute>
 0000:00000000       __hybrid_image_info_bitfield 0000000000000000     <absolute>
 0000:00000000       __x64_code_ranges_to_entry_points 0000000000000000     <absolute>
 0000:00000000       __x64_code_ranges_to_entry_points_count 0000000000000000     <absolute>
 0000:00000100       __guard_flags              0000000000000100     <absolute>
 0000:00000000       __ImageBase                0000000180000000     <linker-defined>
 0001:00000000       Java_sun_security_jgss_wrapper_GSSLibStub_acceptContext 0000000180001000 f   GSSLibStub.obj
 0001:00000724       Java_sun_security_jgss_wrapper_GSSLibStub_acquireCred 0000000180001724 f   GSSLibStub.obj
 0001:000008d8       Java_sun_security_jgss_wrapper_GSSLibStub_canonicalizeName 00000001800018d8 f   GSSLibStub.obj
 0001:000009fc       Java_sun_security_jgss_wrapper_GSSLibStub_compareName 00000001800019fc f   GSSLibStub.obj
 0001:00000ab8       Java_sun_security_jgss_wrapper_GSSLibStub_deleteContext 0000000180001ab8 f   GSSLibStub.obj
 0001:00000b80       Java_sun_security_jgss_wrapper_GSSLibStub_displayName 0000000180001b80 f   GSSLibStub.obj
 0001:00000d3c       Java_sun_security_jgss_wrapper_GSSLibStub_exportContext 0000000180001d3c f   GSSLibStub.obj
 0001:00000e54       Java_sun_security_jgss_wrapper_GSSLibStub_exportName 0000000180001e54 f   GSSLibStub.obj
 0001:0000100c       Java_sun_security_jgss_wrapper_GSSLibStub_getContextMech 000000018000200c f   GSSLibStub.obj
 0001:000010f0       Java_sun_security_jgss_wrapper_GSSLibStub_getContextName 00000001800020f0 f   GSSLibStub.obj
 0001:00001240       Java_sun_security_jgss_wrapper_GSSLibStub_getContextTime 0000000180002240 f   GSSLibStub.obj
 0001:0000131c       Java_sun_security_jgss_wrapper_GSSLibStub_getCredName 000000018000231c f   GSSLibStub.obj
 0001:00001404       Java_sun_security_jgss_wrapper_GSSLibStub_getCredTime 0000000180002404 f   GSSLibStub.obj
 0001:000014ac       Java_sun_security_jgss_wrapper_GSSLibStub_getCredUsage 00000001800024ac f   GSSLibStub.obj
 0001:0000154c       Java_sun_security_jgss_wrapper_GSSLibStub_getMechPtr 000000018000254c f   GSSLibStub.obj
 0001:00001654       Java_sun_security_jgss_wrapper_GSSLibStub_getMic 0000000180002654 f   GSSLibStub.obj
 0001:000017a8       Java_sun_security_jgss_wrapper_GSSLibStub_importContext 00000001800027a8 f   GSSLibStub.obj
 0001:000019c0       Java_sun_security_jgss_wrapper_GSSLibStub_importName 00000001800029c0 f   GSSLibStub.obj
 0001:00001b34       Java_sun_security_jgss_wrapper_GSSLibStub_indicateMechs 0000000180002b34 f   GSSLibStub.obj
 0001:00001b4c       Java_sun_security_jgss_wrapper_GSSLibStub_init 0000000180002b4c f   GSSLibStub.obj
 0001:00001d30       Java_sun_security_jgss_wrapper_GSSLibStub_initContext 0000000180002d30 f   GSSLibStub.obj
 0001:00002164       Java_sun_security_jgss_wrapper_GSSLibStub_inquireContext 0000000180003164 f   GSSLibStub.obj
 0001:0000234c       Java_sun_security_jgss_wrapper_GSSLibStub_inquireNamesForMech 000000018000334c f   GSSLibStub.obj
 0001:00002414       Java_sun_security_jgss_wrapper_GSSLibStub_releaseCred 0000000180003414 f   GSSLibStub.obj
 0001:000024dc       Java_sun_security_jgss_wrapper_GSSLibStub_releaseName 00000001800034dc f   GSSLibStub.obj
 0001:00002588       Java_sun_security_jgss_wrapper_GSSLibStub_unwrap 0000000180003588 f   GSSLibStub.obj
 0001:00002788       Java_sun_security_jgss_wrapper_GSSLibStub_verifyMic 0000000180003788 f   GSSLibStub.obj
 0001:00002968       Java_sun_security_jgss_wrapper_GSSLibStub_wrap 0000000180003968 f   GSSLibStub.obj
 0001:00002b70       Java_sun_security_jgss_wrapper_GSSLibStub_wrapSizeLimit 0000000180003b70 f   GSSLibStub.obj
 0001:00002c78       __local_stdio_printf_options 0000000180003c78 f i GSSLibStub.obj
 0001:00002c80       deleteGSSCB                0000000180003c80 f   GSSLibStub.obj
 0001:00002cdc       fprintf                    0000000180003cdc f i GSSLibStub.obj
 0001:00002d20       inquireCred                0000000180003d20 f   GSSLibStub.obj
 0001:00002e38       newGSSCB                   0000000180003e38 f   GSSLibStub.obj
 0001:00003018       setSupplementaryInfo       0000000180004018 f   GSSLibStub.obj
 0001:000030cc       loadNative                 00000001800040cc f   NativeFunc.obj
 0001:000035c8       JNI_OnLoad                 00000001800045c8 f   NativeUtil.obj
 0001:00003fec       JNI_OnUnload               0000000180004fec f   NativeUtil.obj
 0001:000040a4       checkStatus                00000001800050a4 f   NativeUtil.obj
 0001:0000426c       deleteGSSOID               000000018000526c f   NativeUtil.obj
 0001:00004294       deleteGSSOIDSet            0000000180005294 f   NativeUtil.obj
 0001:000042c4       getGSSTime                 00000001800052c4 f   NativeUtil.obj
 0001:000042d4       getJavaBuffer              00000001800052d4 f   NativeUtil.obj
 0001:00004374       getJavaErrorCode           0000000180005374 f   NativeUtil.obj
 0001:000043b8       getJavaOID                 00000001800053b8 f   NativeUtil.obj
 0001:000044bc       getJavaOIDArray            00000001800054bc f   NativeUtil.obj
 0001:00004594       getJavaString              0000000180005594 f   NativeUtil.obj
 0001:00004660       getJavaTime                0000000180005660 f   NativeUtil.obj
 0001:00004678       getMinorMessage            0000000180005678 f   NativeUtil.obj
 0001:000046ec       gssThrowOutOfMemoryError   00000001800056ec f   NativeUtil.obj
 0001:0000472c       initGSSBuffer              000000018000572c f   NativeUtil.obj
 0001:000047d8       newGSSOID                  00000001800057d8 f   NativeUtil.obj
 0001:000048d0       newGSSOIDSet               00000001800058d0 f   NativeUtil.obj
 0001:00004940       resetGSSBuffer             0000000180005940 f   NativeUtil.obj
 0001:00004968       sameMech                   0000000180005968 f   NativeUtil.obj
 0001:00004994       __GSHandlerCheck           0000000180005994 f   MSVCRT:gshandler.obj
 0001:000049b4       __GSHandlerCheckCommon     00000001800059b4 f   MSVCRT:gshandler.obj
 0001:00004a20       __security_check_cookie    0000000180005a20 f   MSVCRT:amdsecgs.obj
 0001:00004d50       _DllMainCRTStartup         0000000180005d50 f   MSVCRT:dll_dllmain.obj
 0001:00004d90       __raise_securityfailure    0000000180005d90 f   MSVCRT:gs_report.obj
 0001:00004dc4       __report_gsfailure         0000000180005dc4 f   MSVCRT:gs_report.obj
 0001:00004f0c       __security_init_cookie     0000000180005f0c f   MSVCRT:gs_support.obj
 0001:00004fb8       DllMain                    0000000180005fb8 f   MSVCRT:dll_dllmain_stub.obj
 0001:00004fdc       ?__scrt_initialize_type_info@@YAXXZ 0000000180005fdc f   MSVCRT:tncleanup.obj
 0001:00004fec       ?__scrt_uninitialize_type_info@@YAXXZ 0000000180005fec f   MSVCRT:tncleanup.obj
 0001:00004ff8       __local_stdio_scanf_options 0000000180005ff8 f i MSVCRT:default_local_stdio_options.obj
 0001:00005000       __scrt_initialize_default_local_stdio_options 0000000180006000 f   MSVCRT:default_local_stdio_options.obj
 0001:0000501c       __scrt_acquire_startup_lock 000000018000601c f   MSVCRT:utility.obj
 0001:00005058       __scrt_dllmain_after_initialize_c 0000000180006058 f   MSVCRT:utility.obj
 0001:0000508c       __scrt_dllmain_before_initialize_c 000000018000608c f   MSVCRT:utility.obj
 0001:000050a4       __scrt_dllmain_crt_thread_attach 00000001800060a4 f   MSVCRT:utility.obj
 0001:000050cc       __scrt_dllmain_crt_thread_detach 00000001800060cc f   MSVCRT:utility.obj
 0001:000050e4       __scrt_dllmain_exception_filter 00000001800060e4 f   MSVCRT:utility.obj
 0001:00005144       __scrt_dllmain_uninitialize_c 0000000180006144 f   MSVCRT:utility.obj
 0001:00005174       __scrt_dllmain_uninitialize_critical 0000000180006174 f   MSVCRT:utility.obj
 0001:00005188       __scrt_initialize_crt      0000000180006188 f   MSVCRT:utility.obj
 0001:000051c4       __scrt_initialize_onexit_tables 00000001800061c4 f   MSVCRT:utility.obj
 0001:00005250       __scrt_is_nonwritable_in_current_image 0000000180006250 f   MSVCRT:utility.obj
 0001:000052e8       __scrt_release_startup_lock 00000001800062e8 f   MSVCRT:utility.obj
 0001:0000530c       __scrt_uninitialize_crt    000000018000630c f   MSVCRT:utility.obj
 0001:00005338       __scrt_get_dyn_tls_init_callback 0000000180006338 f   MSVCRT:dyn_tls_init.obj
 0001:00005340       __crt_debugger_hook        0000000180006340 f   MSVCRT:utility_desktop.obj
 0001:00005348       __scrt_fastfail            0000000180006348 f   MSVCRT:utility_desktop.obj
 0001:00005490       _RTC_Initialize            0000000180006490 f   MSVCRT:initsect.obj
 0001:000054cc       _RTC_Terminate             00000001800064cc f   MSVCRT:initsect.obj
 0001:00005508       _guard_check_icall_nop     0000000180006508 f i MSVCRT:guard_support.obj
 0001:0000550c       __isa_available_init       000000018000650c f   MSVCRT:cpu_disp.obj
 0001:000057d8       _get_startup_argv_mode     00000001800067d8 f   MSVCRT:argv_mode.obj
 0001:000057e0       __scrt_is_ucrt_dll_in_use  00000001800067e0 f   MSVCRT:ucrt_detection.obj
 0001:000057f0       memcmp                     00000001800067f0 f   vcruntime:VCRUNTIME140.dll
 0001:000057f6       __C_specific_handler       00000001800067f6 f   vcruntime:VCRUNTIME140.dll
 0001:000057fc       __std_type_info_destroy_list 00000001800067fc f   vcruntime:VCRUNTIME140.dll
 0001:00005802       memset                     0000000180006802 f   vcruntime:VCRUNTIME140.dll
 0001:00005808       _initterm                  0000000180006808 f   ucrt:api-ms-win-crt-runtime-l1-1-0.dll
 0001:0000580e       _initterm_e                000000018000680e f   ucrt:api-ms-win-crt-runtime-l1-1-0.dll
 0001:00005814       _seh_filter_dll            0000000180006814 f   ucrt:api-ms-win-crt-runtime-l1-1-0.dll
 0001:0000581a       _configure_narrow_argv     000000018000681a f   ucrt:api-ms-win-crt-runtime-l1-1-0.dll
 0001:00005820       _initialize_narrow_environment 0000000180006820 f   ucrt:api-ms-win-crt-runtime-l1-1-0.dll
 0001:00005826       _initialize_onexit_table   0000000180006826 f   ucrt:api-ms-win-crt-runtime-l1-1-0.dll
 0001:0000582c       _execute_onexit_table      000000018000682c f   ucrt:api-ms-win-crt-runtime-l1-1-0.dll
 0001:00005832       _cexit                     0000000180006832 f   ucrt:api-ms-win-crt-runtime-l1-1-0.dll
 0001:00005838       __acrt_initialize          0000000180006838 f   MSVCRT:ucrt_stubs.obj
 0001:00005838       __acrt_thread_attach       0000000180006838 f   MSVCRT:ucrt_stubs.obj
 0001:00005838       __acrt_thread_detach       0000000180006838 f   MSVCRT:ucrt_stubs.obj
 0001:00005838       __acrt_uninitialize        0000000180006838 f   MSVCRT:ucrt_stubs.obj
 0001:00005838       __acrt_uninitialize_critical 0000000180006838 f   MSVCRT:ucrt_stubs.obj
 0001:00005838       __scrt_stub_for_acrt_initialize 0000000180006838 f   MSVCRT:ucrt_stubs.obj
 0001:00005838       __scrt_stub_for_acrt_thread_attach 0000000180006838 f   MSVCRT:ucrt_stubs.obj
 0001:00005838       __scrt_stub_for_acrt_thread_detach 0000000180006838 f   MSVCRT:ucrt_stubs.obj
 0001:00005838       __scrt_stub_for_acrt_uninitialize 0000000180006838 f   MSVCRT:ucrt_stubs.obj
 0001:00005838       __scrt_stub_for_acrt_uninitialize_critical 0000000180006838 f   MSVCRT:ucrt_stubs.obj
 0001:00005838       __vcrt_initialize          0000000180006838 f   MSVCRT:ucrt_stubs.obj
 0001:00005838       __vcrt_thread_attach       0000000180006838 f   MSVCRT:ucrt_stubs.obj
 0001:00005838       __vcrt_thread_detach       0000000180006838 f   MSVCRT:ucrt_stubs.obj
 0001:00005838       __vcrt_uninitialize        0000000180006838 f   MSVCRT:ucrt_stubs.obj
 0001:00005838       __vcrt_uninitialize_critical 0000000180006838 f   MSVCRT:ucrt_stubs.obj
 0001:0000583c       __scrt_stub_for_is_c_termination_complete 000000018000683c f   MSVCRT:ucrt_stubs.obj
 0001:0000583c       _is_c_termination_complete 000000018000683c f   MSVCRT:ucrt_stubs.obj
 0001:0000583f       memcpy                     000000018000683f f   vcruntime:VCRUNTIME140.dll
 0001:00005860       _guard_dispatch_icall_nop  0000000180006860 f   MSVCRT:guard_dispatch.obj
 0001:00005880       _guard_xfg_dispatch_icall_nop 0000000180006880 f   MSVCRT:guard_xfg_dispatch.obj
 0002:00000000       __imp_GetLastError         0000000180007000     kernel32:KERNEL32.dll
 0002:00000008       __imp_FormatMessageA       0000000180007008     kernel32:KERNEL32.dll
 0002:00000010       __imp_CloseHandle          0000000180007010     kernel32:KERNEL32.dll
 0002:00000018       __imp_GetProcAddress       0000000180007018     kernel32:KERNEL32.dll
 0002:00000020       __imp_LoadLibraryA         0000000180007020     kernel32:KERNEL32.dll
 0002:00000028       __imp_RtlCaptureContext    0000000180007028     kernel32:KERNEL32.dll
 0002:00000030       __imp_RtlLookupFunctionEntry 0000000180007030     kernel32:KERNEL32.dll
 0002:00000038       __imp_RtlVirtualUnwind     0000000180007038     kernel32:KERNEL32.dll
 0002:00000040       __imp_UnhandledExceptionFilter 0000000180007040     kernel32:KERNEL32.dll
 0002:00000048       __imp_SetUnhandledExceptionFilter 0000000180007048     kernel32:KERNEL32.dll
 0002:00000050       __imp_GetCurrentProcess    0000000180007050     kernel32:KERNEL32.dll
 0002:00000058       __imp_TerminateProcess     0000000180007058     kernel32:KERNEL32.dll
 0002:00000060       __imp_IsProcessorFeaturePresent 0000000180007060     kernel32:KERNEL32.dll
 0002:00000068       __imp_QueryPerformanceCounter 0000000180007068     kernel32:KERNEL32.dll
 0002:00000070       __imp_GetCurrentProcessId  0000000180007070     kernel32:KERNEL32.dll
 0002:00000078       __imp_GetCurrentThreadId   0000000180007078     kernel32:KERNEL32.dll
 0002:00000080       __imp_GetSystemTimeAsFileTime 0000000180007080     kernel32:KERNEL32.dll
 0002:00000088       __imp_DisableThreadLibraryCalls 0000000180007088     kernel32:KERNEL32.dll
 0002:00000090       __imp_InitializeSListHead  0000000180007090     kernel32:KERNEL32.dll
 0002:00000098       __imp_IsDebuggerPresent    0000000180007098     kernel32:KERNEL32.dll
 0002:000000a0       \177KERNEL32_NULL_THUNK_DATA 00000001800070a0     kernel32:KERNEL32.dll
 0002:000000a8       __imp_memcmp               00000001800070a8     vcruntime:VCRUNTIME140.dll
 0002:000000b0       __imp___C_specific_handler 00000001800070b0     vcruntime:VCRUNTIME140.dll
 0002:000000b8       __imp___std_type_info_destroy_list 00000001800070b8     vcruntime:VCRUNTIME140.dll
 0002:000000c0       __imp_memset               00000001800070c0     vcruntime:VCRUNTIME140.dll
 0002:000000c8       __imp_memcpy               00000001800070c8     vcruntime:VCRUNTIME140.dll
 0002:000000d0       \177VCRUNTIME140_NULL_THUNK_DATA 00000001800070d0     vcruntime:VCRUNTIME140.dll
 0002:000000d8       __imp_free                 00000001800070d8     ucrt:api-ms-win-crt-heap-l1-1-0.dll
 0002:000000e0       __imp_calloc               00000001800070e0     ucrt:api-ms-win-crt-heap-l1-1-0.dll
 0002:000000e8       __imp_malloc               00000001800070e8     ucrt:api-ms-win-crt-heap-l1-1-0.dll
 0002:000000f0       \177api-ms-win-crt-heap-l1-1-0_NULL_THUNK_DATA 00000001800070f0     ucrt:api-ms-win-crt-heap-l1-1-0.dll
 0002:000000f8       __imp__initialize_onexit_table 00000001800070f8     ucrt:api-ms-win-crt-runtime-l1-1-0.dll
 0002:00000100       __imp__initterm            0000000180007100     ucrt:api-ms-win-crt-runtime-l1-1-0.dll
 0002:00000108       __imp__initterm_e          0000000180007108     ucrt:api-ms-win-crt-runtime-l1-1-0.dll
 0002:00000110       __imp__seh_filter_dll      0000000180007110     ucrt:api-ms-win-crt-runtime-l1-1-0.dll
 0002:00000118       __imp__configure_narrow_argv 0000000180007118     ucrt:api-ms-win-crt-runtime-l1-1-0.dll
 0002:00000120       __imp__initialize_narrow_environment 0000000180007120     ucrt:api-ms-win-crt-runtime-l1-1-0.dll
 0002:00000128       __imp__execute_onexit_table 0000000180007128     ucrt:api-ms-win-crt-runtime-l1-1-0.dll
 0002:00000130       __imp__cexit               0000000180007130     ucrt:api-ms-win-crt-runtime-l1-1-0.dll
 0002:00000138       \177api-ms-win-crt-runtime-l1-1-0_NULL_THUNK_DATA 0000000180007138     ucrt:api-ms-win-crt-runtime-l1-1-0.dll
 0002:00000140       __imp___stdio_common_vfprintf 0000000180007140     ucrt:api-ms-win-crt-stdio-l1-1-0.dll
 0002:00000148       __imp_fflush               0000000180007148     ucrt:api-ms-win-crt-stdio-l1-1-0.dll
 0002:00000150       __imp___acrt_iob_func      0000000180007150     ucrt:api-ms-win-crt-stdio-l1-1-0.dll
 0002:00000158       \177api-ms-win-crt-stdio-l1-1-0_NULL_THUNK_DATA 0000000180007158     ucrt:api-ms-win-crt-stdio-l1-1-0.dll
 0002:00000160       __guard_check_icall_fptr   0000000180007160     MSVCRT:guard_support.obj
 0002:00000168       __guard_xfg_check_icall_fptr 0000000180007168     MSVCRT:guard_support.obj
 0002:00000170       __guard_dispatch_icall_fptr 0000000180007170     MSVCRT:guard_support.obj
 0002:00000178       __guard_xfg_dispatch_icall_fptr 0000000180007178     MSVCRT:guard_support.obj
 0002:00000180       __guard_xfg_table_dispatch_icall_fptr 0000000180007180     MSVCRT:guard_support.obj
 0002:00000188       __castguard_check_failure_os_handled_fptr 0000000180007188     MSVCRT:guard_support.obj
 0002:00000190       __guard_memcpy_fptr        0000000180007190     vcruntime:softmemtag.obj
 0002:00000198       __xc_a                     0000000180007198     MSVCRT:initializers.obj
 0002:000001a0       __xc_z                     00000001800071a0     MSVCRT:initializers.obj
 0002:000001a8       __xi_a                     00000001800071a8     MSVCRT:initializers.obj
 0002:000001b0       __xi_z                     00000001800071b0     MSVCRT:initializers.obj
 0002:000001b8       __xp_a                     00000001800071b8     MSVCRT:initializers.obj
 0002:000001c0       __xp_z                     00000001800071c0     MSVCRT:initializers.obj
 0002:000001c8       __xt_a                     00000001800071c8     MSVCRT:initializers.obj
 0002:000001d0       __xt_z                     00000001800071d0     MSVCRT:initializers.obj
 0002:000001e0       TYPE_CRED_NAME             00000001800071e0     GSSLibStub.obj
 0002:000001e4       TYPE_CRED_TIME             00000001800071e4     GSSLibStub.obj
 0002:000001e8       TYPE_CRED_USAGE            00000001800071e8     GSSLibStub.obj
 0002:000001f0       ??_C@_0CH@IFIMLFDG@?$FLGSSLibStub_init?$FN?5GSS?5lib?5name?5@ 00000001800071f0     GSSLibStub.obj
 0002:00000218       ??_C@_0BE@FBKICJJF@?$FLGSSLibStub?3?$CFd?$FN?5?$CFs?6@ 0000000180007218     GSSLibStub.obj
 0002:00000230       ??_C@_0CO@DHBKBJOL@?$FLGSSLibStub?3?$CFd?$FN?5?$FLGSSLibStub_ini@ 0000000180007230     GSSLibStub.obj
 0002:00000260       ??_C@_0DG@BBGFBBEA@sun?1security?1jgss?1krb5?1internal@ 0000000180007260     GSSLibStub.obj
 0002:00000298       ??_C@_0CN@IGOHGPID@?$FLGSSLibStub?3?$CFd?$FN?5GSS?9API?3?5Unknow@ 0000000180007298     GSSLibStub.obj
 0002:000002c8       ??_C@_0BN@IKLFJBD@?$FLGSSLibStub?3?$CFd?$FN?5GSS?9API?3?5?$CFs?6@ 00000001800072c8     GSSLibStub.obj
 0002:000002e8       ??_C@_0BI@FIIPHNCE@?$FLGSSLibStub_getMechPtr?$FN@ 00000001800072e8     GSSLibStub.obj
 0002:00000300       ??_C@_0CB@EEKJDBHK@?$FLGSSLibStub_inquireNamesForMech@ 0000000180007300     GSSLibStub.obj
 0002:00000328       ??_C@_0CO@FNFLNOMG@?$FLGSSLibStub?3?$CFd?$FN?5?$FLGSSLibStub_rel@ 0000000180007328     GSSLibStub.obj
 0002:00000358       ??_C@_0BJ@CBIHLCMJ@?$FLGSSLibStub_releaseName?$FN@ 0000000180007358     GSSLibStub.obj
 0002:00000378       ??_C@_0BI@DFKAFKP@?$FLGSSLibStub_importName?$FN@ 0000000180007378     GSSLibStub.obj
 0002:00000390       ??_C@_0CO@DHOLOMBP@?$FLGSSLibStub?3?$CFd?$FN?5?$FLGSSLibStub_imp@ 0000000180007390     GSSLibStub.obj
 0002:000003c0       ??_C@_0DC@EDJDCFOA@?$FLGSSLibStub?3?$CFd?$FN?5?$FLGSSLibStub_com@ 00000001800073c0     GSSLibStub.obj
 0002:000003f8       ??_C@_0BJ@GOICLAAF@?$FLGSSLibStub_compareName?$FN@ 00000001800073f8     GSSLibStub.obj
 0002:00000418       ??_C@_0DD@PNOHLKNJ@?$FLGSSLibStub?3?$CFd?$FN?5?$FLGSSLibStub_can@ 0000000180007418     GSSLibStub.obj
 0002:00000450       ??_C@_0DH@NIBOKLIJ@?$FLGSSLibStub?3?$CFd?$FN?5?$FLGSSLibStub_can@ 0000000180007450     GSSLibStub.obj
 0002:00000488       ??_C@_0BO@MEBIAJAG@?$FLGSSLibStub_canonicalizeName?$FN@ 0000000180007488     GSSLibStub.obj
 0002:000004a8       ??_C@_0CN@HMNALJKN@?$FLGSSLibStub?3?$CFd?$FN?5?$FLGSSLibStub_exp@ 00000001800074a8     GSSLibStub.obj
 0002:000004d8       ??_C@_0DA@BMLGEALK@?$FLGSSLibStub_exportName?$FN?5canonic@ 00000001800074d8     GSSLibStub.obj
 0002:00000508       ??_C@_0BI@NJPBCAKH@?$FLGSSLibStub_exportName?$FN@ 0000000180007508     GSSLibStub.obj
 0002:00000520       ??_C@_0CO@JNAHONNN@?$FLGSSLibStub?3?$CFd?$FN?5?$FLGSSLibStub_dis@ 0000000180007520     GSSLibStub.obj
 0002:00000550       ??_C@_0BJ@KDEJNLFF@?$FLGSSLibStub_displayName?$FN@ 0000000180007550     GSSLibStub.obj
 0002:00000570       ??_C@_0BJ@KNGBMLML@?$FLGSSLibStub_acquireCred?$FN@ 0000000180007570     GSSLibStub.obj
 0002:00000590       ??_C@_0DO@GCCNNHHE@?$FLGSSLibStub?3?$CFd?$FN?5?$FLGSSLibStub_acq@ 0000000180007590     GSSLibStub.obj
 0002:000005d0       ??_C@_0DF@HFNBAFII@?$FLGSSLibStub?3?$CFd?$FN?5?$FLGSSLibStub_acq@ 00000001800075d0     GSSLibStub.obj
 0002:00000608       ??_C@_0CO@CNCEALKM@?$FLGSSLibStub?3?$CFd?$FN?5?$FLGSSLibStub_rel@ 0000000180007608     GSSLibStub.obj
 0002:00000638       ??_C@_0BJ@HOCPAOJN@?$FLGSSLibStub_releaseCred?$FN@ 0000000180007638     GSSLibStub.obj
 0002:00000658       ??_C@_0CJ@IINKCHDK@?$FLGSSLibStub?3?$CFd?$FN?5?$FLgss_inquire_cr@ 0000000180007658     GSSLibStub.obj
 0002:00000688       ??_C@_0BD@NFEKOCFD@?$FLgss_inquire_cred?$FN@ 0000000180007688     GSSLibStub.obj
 0002:000006a0       ??_C@_0CO@DNJNIEFL@?$FLGSSLibStub?3?$CFd?$FN?5?$FLGSSLibStub_get@ 00000001800076a0     GSSLibStub.obj
 0002:000006d0       ??_C@_0DF@KIBOHKHD@?$FLGSSLibStub?3?$CFd?$FN?5?$FLGSSLibStub_get@ 00000001800076d0     GSSLibStub.obj
 0002:00000708       ??_C@_0CO@GCBDFIOA@?$FLGSSLibStub?3?$CFd?$FN?5?$FLGSSLibStub_get@ 0000000180007708     GSSLibStub.obj
 0002:00000738       ??_C@_0CP@OAPFJNOP@?$FLGSSLibStub?3?$CFd?$FN?5?$FLGSSLibStub_get@ 0000000180007738     GSSLibStub.obj
 0002:00000768       ??_C@_0BL@FKHNPAJG@?$FLGSSLibStub_importContext?$FN@ 0000000180007768     GSSLibStub.obj
 0002:00000788       ??_C@_0DK@KFHKDMPI@?$FLGSSLibStub?3?$CFd?$FN?5?$FLGSSLibStub_imp@ 0000000180007788     GSSLibStub.obj
 0002:000007c8       ??_C@_0CD@BCECEGFB@?$FLGSSLibStub_importContext?$FN?5getM@ 00000001800077c8     GSSLibStub.obj
 0002:000007f0       ??_C@_0CD@ICJKNONJ@?$FLGSSLibStub_importContext?$FN?5clea@ 00000001800077f0     GSSLibStub.obj
 0002:00000818       ??_C@_0BJ@BFLGHPHA@?$FLGSSLibStub_initContext?$FN@ 0000000180007818     GSSLibStub.obj
 0002:00000840       ??_C@_0EM@MFMNDJHA@?$FLGSSLibStub?3?$CFd?$FN?5?$FLGSSLibStub_ini@ 0000000180007840     GSSLibStub.obj
 0002:00000890       ??_C@_0FB@BBCFOABH@?$FLGSSLibStub?3?$CFd?$FN?5?$FLGSSLibStub_ini@ 0000000180007890     GSSLibStub.obj
 0002:000008e8       ??_C@_0DM@IHCDOPFD@?$FLGSSLibStub?3?$CFd?$FN?5?$FLGSSLibStub_ini@ 00000001800078e8     GSSLibStub.obj
 0002:00000928       ??_C@_0DJ@EHOIIEEF@?$FLGSSLibStub?3?$CFd?$FN?5?$FLGSSLibStub_ini@ 0000000180007928     GSSLibStub.obj
 0002:00000968       ??_C@_0CN@EFAHJDCF@?$FLGSSLibStub_initContext?$FN?5contex@ 0000000180007968     GSSLibStub.obj
 0002:00000998       ??_C@_0DB@LEECDODG@?$FLGSSLibStub_initContext?$FN?5contex@ 0000000180007998     GSSLibStub.obj
 0002:000009d0       ??_C@_0BL@OFPJPCCF@?$FLGSSLibStub_acceptContext?$FN@ 00000001800079d0     GSSLibStub.obj
 0002:000009f0       ??_C@_0EO@DHNGKIO@?$FLGSSLibStub?3?$CFd?$FN?5?$FLGSSLibStub_acc@ 00000001800079f0     GSSLibStub.obj
 0002:00000a40       ??_C@_0FO@KEIFGJNP@?$FLGSSLibStub?3?$CFd?$FN?5?$FLGSSLibStub_acc@ 0000000180007a40     GSSLibStub.obj
 0002:00000aa0       ??_C@_0DO@FLOPEGOD@?$FLGSSLibStub?3?$CFd?$FN?5?$FLGSSLibStub_acc@ 0000000180007aa0     GSSLibStub.obj
 0002:00000ae0       ??_C@_0DL@FNMHCNEI@?$FLGSSLibStub?3?$CFd?$FN?5?$FLGSSLibStub_acc@ 0000000180007ae0     GSSLibStub.obj
 0002:00000b20       ??_C@_0CD@POJPGDLJ@?$FLGSSLibStub_acceptContext?$FN?5inqu@ 0000000180007b20     GSSLibStub.obj
 0002:00000b50       ??_C@_0EA@MNGHEEKJ@?$FLGSSLibStub?3?$CFd?$FN?5?$FLGSSLibStub_acc@ 0000000180007b50     GSSLibStub.obj
 0002:00000b90       ??_C@_0DN@LJGBHPGK@?$FLGSSLibStub?3?$CFd?$FN?5?$FLGSSLibStub_acc@ 0000000180007b90     GSSLibStub.obj
 0002:00000bd0       ??_C@_0CP@IEEDNBPF@?$FLGSSLibStub_acceptContext?$FN?5cont@ 0000000180007bd0     GSSLibStub.obj
 0002:00000c00       ??_C@_0ED@OFFGMJFO@?$FLGSSLibStub?3?$CFd?$FN?5?$FLGSSLibStub_acc@ 0000000180007c00     GSSLibStub.obj
 0002:00000c48       ??_C@_0DD@JJHOKGCG@?$FLGSSLibStub_acceptContext?$FN?5cont@ 0000000180007c48     GSSLibStub.obj
 0002:00000c80       ??_C@_0DC@PADJEPMC@?$FLGSSLibStub?3?$CFd?$FN?5?$FLGSSLibStub_inq@ 0000000180007c80     GSSLibStub.obj
 0002:00000cc0       ??_C@_0EL@GELLJEOM@?$FLGSSLibStub?3?$CFd?$FN?5?$FLGSSLibStub_inq@ 0000000180007cc0     GSSLibStub.obj
 0002:00000d10       ??_C@_0BM@IFAECBDO@?$FLGSSLibStub_inquireContext?$FN@ 0000000180007d10     GSSLibStub.obj
 0002:00000d30       ??_C@_0DB@IFOABMAJ@?$FLGSSLibStub?3?$CFd?$FN?5?$FLGSSLibStub_get@ 0000000180007d30     GSSLibStub.obj
 0002:00000d68       ??_C@_0BM@COJKOILK@?$FLGSSLibStub_getContextMech?$FN@ 0000000180007d68     GSSLibStub.obj
 0002:00000d88       ??_C@_0DM@OGJELJAI@?$FLGSSLibStub?3?$CFd?$FN?5?$FLGSSLibStub_get@ 0000000180007d88     GSSLibStub.obj
 0002:00000dc8       ??_C@_0BP@DPDPDKIA@?$FLGSSLibStub_inquireContextAll?$FN@ 0000000180007dc8     GSSLibStub.obj
 0002:00000de8       ??_C@_0DI@HBOHCKMC@?$FLGSSLibStub?3?$CFd?$FN?5?$FLGSSLibStub_get@ 0000000180007de8     GSSLibStub.obj
 0002:00000e20       ??_C@_0DC@GNICCFPO@?$FLGSSLibStub?3?$CFd?$FN?5?$FLGSSLibStub_get@ 0000000180007e20     GSSLibStub.obj
 0002:00000e58       ??_C@_0BM@CHLELCII@?$FLGSSLibStub_getContextTime?$FN@ 0000000180007e58     GSSLibStub.obj
 0002:00000e78       ??_C@_0DB@KAKCNCBB@?$FLGSSLibStub?3?$CFd?$FN?5?$FLGSSLibStub_del@ 0000000180007e78     GSSLibStub.obj
 0002:00000eb0       ??_C@_0BL@HBHJELHJ@?$FLGSSLibStub_deleteContext?$FN@ 0000000180007eb0     GSSLibStub.obj
 0002:00000ed0       ??_C@_0DB@JOGDAKAL@?$FLGSSLibStub?3?$CFd?$FN?5?$FLGSSLibStub_wra@ 0000000180007ed0     GSSLibStub.obj
 0002:00000f08       ??_C@_0BL@GNPIIACB@?$FLGSSLibStub_wrapSizeLimit?$FN@ 0000000180007f08     GSSLibStub.obj
 0002:00000f28       ??_C@_0DB@GHJKAKOC@?$FLGSSLibStub?3?$CFd?$FN?5?$FLGSSLibStub_exp@ 0000000180007f28     GSSLibStub.obj
 0002:00000f60       ??_C@_0BL@PNJJALHD@?$FLGSSLibStub_exportContext?$FN@ 0000000180007f60     GSSLibStub.obj
 0002:00000f80       ??_C@_0CK@IGOIEBFN@?$FLGSSLibStub?3?$CFd?$FN?5?$FLGSSLibStub_get@ 0000000180007f80     GSSLibStub.obj
 0002:00000fb0       ??_C@_0BE@PDIMELDO@?$FLGSSLibStub_getMic?$FN@ 0000000180007fb0     GSSLibStub.obj
 0002:00000fc8       ??_C@_0CN@OMIJFGJO@?$FLGSSLibStub?3?$CFd?$FN?5?$FLGSSLibStub_ver@ 0000000180007fc8     GSSLibStub.obj
 0002:00000ff8       ??_C@_0BH@IPGHLHPO@?$FLGSSLibStub_verifyMic?$FN@ 0000000180007ff8     GSSLibStub.obj
 0002:00001010       ??_C@_0CI@IALAIHOK@?$FLGSSLibStub?3?$CFd?$FN?5?$FLGSSLibStub_wra@ 0000000180008010     GSSLibStub.obj
 0002:00001038       ??_C@_0BC@HKCNLDAH@?$FLGSSLibStub_wrap?$FN@ 0000000180008038     GSSLibStub.obj
 0002:00001050       ??_C@_0CK@KMGLFFFF@?$FLGSSLibStub?3?$CFd?$FN?5?$FLGSSLibStub_unw@ 0000000180008050     GSSLibStub.obj
 0002:00001080       ??_C@_0BE@LBCEEBKN@?$FLGSSLibStub_unwrap?$FN@ 0000000180008080     GSSLibStub.obj
 0002:00001320       JAVA_DUPLICATE_TOKEN_CODE  0000000180008320     NativeUtil.obj
 0002:00001324       JAVA_OLD_TOKEN_CODE        0000000180008324     NativeUtil.obj
 0002:00001328       JAVA_UNSEQ_TOKEN_CODE      0000000180008328     NativeUtil.obj
 0002:0000132c       JAVA_GAP_TOKEN_CODE        000000018000832c     NativeUtil.obj
 0002:00001330       JAVA_ERROR_CODE            0000000180008330     NativeUtil.obj
 0002:00001378       SPNEGO_BYTES               0000000180008378     NativeUtil.obj
 0002:00001380       JAVA_MAX                   0000000180008380     NativeUtil.obj
 0002:00001388       ??_C@_0BB@DDFKOHA@java?1lang?1Object@ 0000000180008388     NativeUtil.obj
 0002:000013a0       ??_C@_0BM@IGAFBDKG@Couldn?8t?5find?5Object?5class?6@ 00000001800083a0     NativeUtil.obj
 0002:000013c0       ??_C@_0BB@FLFAIHG@java?1lang?1String@ 00000001800083c0     NativeUtil.obj
 0002:000013d8       ??_C@_0BM@LOBNDLCB@Couldn?8t?5find?5String?5class?6@ 00000001800083d8     NativeUtil.obj
 0002:000013f8       ??_C@_0BC@LECFJELF@org?1ietf?1jgss?1Oid@ 00000001800083f8     NativeUtil.obj
 0002:00001410       ??_C@_0CH@PGPGONKK@Couldn?8t?5find?5org?4ietf?4jgss?4Oid@ 0000000180008410     NativeUtil.obj
 0002:00001438       ??_C@_0BL@FNACHLFG@org?1ietf?1jgss?1GSSException@ 0000000180008438     NativeUtil.obj
 0002:00001458       ??_C@_0DA@GFNNKFCG@Couldn?8t?5find?5org?4ietf?4jgss?4GSS@ 0000000180008458     NativeUtil.obj
 0002:00001488       ??_C@_0CJ@MAIAMGJJ@sun?1security?1jgss?1wrapper?1GSSNa@ 0000000180008488     NativeUtil.obj
 0002:000014b8       ??_C@_0DO@BINJABLK@Couldn?8t?5find?5sun?4security?4jgss@ 00000001800084b8     NativeUtil.obj
 0002:000014f8       ??_C@_0CJ@GNJHDBAK@sun?1security?1jgss?1wrapper?1GSSCr@ 00000001800084f8     NativeUtil.obj
 0002:00001528       ??_C@_0DO@KDKPMOPA@Couldn?8t?5find?5sun?4security?4jgss@ 0000000180008528     NativeUtil.obj
 0002:00001568       ??_C@_0CL@KFFCDPKJ@sun?1security?1jgss?1wrapper?1Nativ@ 0000000180008568     NativeUtil.obj
 0002:000015a0       ??_C@_0EA@KEIEKLLE@Couldn?8t?5find?5sun?4security?4jgss@ 00000001800085a0     NativeUtil.obj
 0002:000015e0       ??_C@_0CM@FIPIMGBP@sun?1security?1jgss?1wrapper?1SunNa@ 00000001800085e0     NativeUtil.obj
 0002:00001610       ??_C@_0EB@CKAABFEK@Couldn?8t?5find?5sun?4security?4jgss@ 0000000180008610     NativeUtil.obj
 0002:00001654       ??_C@_05GBDANG@?$CI?$FLB?$CJV@ 0000000180008654     NativeUtil.obj
 0002:0000165c       ??_C@_06FALKBLGB@?$DMinit?$DO@ 000000018000865c     NativeUtil.obj
 0002:00001668       ??_C@_0CK@EGDHFDIO@Couldn?8t?5find?5String?$CIbyte?$FL?$FN?$CJ?5co@ 0000000180008668     NativeUtil.obj
 0002:00001698       ??_C@_0CH@EFPONDAE@Couldn?8t?5find?5Oid?$CIbyte?$FL?$FN?$CJ?5const@ 0000000180008698     NativeUtil.obj
 0002:000016c0       ??_C@_04LHPAGAEF@?$CI?$CJ?$FLB@ 00000001800086c0     NativeUtil.obj
 0002:000016c8       ??_C@_06JCEDDFJL@getDER@   00000001800086c8     NativeUtil.obj
 0002:000016d0       ??_C@_0CD@BPHKINPK@Couldn?8t?5find?5Oid?4getDER?$CI?$CJ?5meth@ 00000001800086d0     NativeUtil.obj
 0002:000016f8       ??_C@_0BK@ECDCMHPE@org?1ietf?1jgss?1MessageProp@ 00000001800086f8     NativeUtil.obj
 0002:00001718       ??_C@_0CP@OAIPCLPB@Couldn?8t?5find?5org?4ietf?4jgss?4Mes@ 0000000180008718     NativeUtil.obj
 0002:00001748       ??_C@_03MMPFGPID@?$CI?$CJZ@ 0000000180008748     NativeUtil.obj
 0002:00001750       ??_C@_0L@DHFIMONM@getPrivacy@ 0000000180008750     NativeUtil.obj
 0002:00001760       ??_C@_0CP@ELGGFPHK@Couldn?8t?5find?5MessageProp?4getPr@ 0000000180008760     NativeUtil.obj
 0002:00001790       ??_C@_03KNBKCOBB@?$CI?$CJI@ 0000000180008790     NativeUtil.obj
 0002:00001794       ??_C@_06MKCFHFGC@getQOP@   0000000180008794     NativeUtil.obj
 0002:000017a0       ??_C@_0CL@HPEKBOID@Couldn?8t?5find?5MessageProp?4getQO@ 00000001800087a0     NativeUtil.obj
 0002:000017cc       ??_C@_04LHKBAEFM@?$CIZ?$CJV@ 00000001800087cc     NativeUtil.obj
 0002:000017d8       ??_C@_0L@CJHHHJJF@setPrivacy@ 00000001800087d8     NativeUtil.obj
 0002:000017e8       ??_C@_0DG@IIGPDELO@Couldn?8t?5find?5MessageProp?4setPr@ 00000001800087e8     NativeUtil.obj
 0002:00001820       ??_C@_04PFANPMCN@?$CII?$CJV@ 0000000180008820     NativeUtil.obj
 0002:00001828       ??_C@_06FJLEMNLP@setQOP@   0000000180008828     NativeUtil.obj
 0002:00001830       ??_C@_0CO@MPIMJBGL@Couldn?8t?5find?5MessageProp?4setQO@ 0000000180008830     NativeUtil.obj
 0002:00001860       ??_C@_0BL@NJFIGAKL@?$CIZZZZILjava?1lang?1String?$DL?$CJV@ 0000000180008860     NativeUtil.obj
 0002:00001880       ??_C@_0BH@MMNNCMHK@setSupplementaryStates@ 0000000180008880     NativeUtil.obj
 0002:00001898       ??_C@_0DO@DMHBAJGD@Couldn?8t?5find?5MessageProp?4setSu@ 0000000180008898     NativeUtil.obj
 0002:000018d8       ??_C@_0BI@GGPJCDGB@?$CIIILjava?1lang?1String?$DL?$CJV@ 00000001800088d8     NativeUtil.obj
 0002:000018f0       ??_C@_0DK@MKODGPFC@Couldn?8t?5find?5GSSException?$CIint?0@ 00000001800088f0     NativeUtil.obj
 0002:00001930       ??_C@_0BN@PCMKHBAM@org?1ietf?1jgss?1ChannelBinding@ 0000000180008930     NativeUtil.obj
 0002:00001950       ??_C@_0DC@KLFKEJOB@Couldn?8t?5find?5org?4ietf?4jgss?4Cha@ 0000000180008950     NativeUtil.obj
 0002:00001988       ??_C@_0BJ@PCBGABPN@?$CI?$CJLjava?1net?1InetAddress?$DL@ 0000000180008988     NativeUtil.obj
 0002:000019a8       ??_C@_0BE@BFCHFIIG@getInitiatorAddress@ 00000001800089a8     NativeUtil.obj
 0002:000019c0       ??_C@_0DL@FKEIDKDF@Couldn?8t?5find?5ChannelBinding?4ge@ 00000001800089c0     NativeUtil.obj
 0002:00001a00       ??_C@_0BD@GABBFHOC@getAcceptorAddress@ 0000000180008a00     NativeUtil.obj
 0002:00001a18       ??_C@_0DK@IABBFOKP@Couldn?8t?5find?5ChannelBinding?4ge@ 0000000180008a18     NativeUtil.obj
 0002:00001a58       ??_C@_0BD@IGFAEMMP@getApplicationData@ 0000000180008a58     NativeUtil.obj
 0002:00001a70       ??_C@_0DK@JBGAFLDN@Couldn?8t?5find?5ChannelBinding?4ge@ 0000000180008a70     NativeUtil.obj
 0002:00001ab0       ??_C@_0BF@LNJHKELF@java?1net?1InetAddress@ 0000000180008ab0     NativeUtil.obj
 0002:00001ac8       ??_C@_0CK@FNACPNDF@Couldn?8t?5find?5java?4net?4InetAddr@ 0000000180008ac8     NativeUtil.obj
 0002:00001af8       ??_C@_0L@KDPCDPCO@getAddress@ 0000000180008af8     NativeUtil.obj
 0002:00001b08       ??_C@_0CP@HGHKJAFB@Couldn?8t?5find?5InetAddress?4getAd@ 0000000180008b08     NativeUtil.obj
 0002:00001b38       ??_C@_0CL@DOONCHMP@?$CIJLsun?1security?1jgss?1wrapper?1GS@ 0000000180008b38     NativeUtil.obj
 0002:00001b68       ??_C@_0DM@MCLCHDAJ@Couldn?8t?5find?5GSSNameElement?$CIlo@ 0000000180008b68     NativeUtil.obj
 0002:00001bb0       ??_C@_0EC@KINGCJOP@?$CIJLsun?1security?1jgss?1wrapper?1GS@ 0000000180008bb0     NativeUtil.obj
 0002:00001bf8       ??_C@_0DM@LOKCAJBC@Couldn?8t?5find?5GSSCredElement?$CIlo@ 0000000180008bf8     NativeUtil.obj
 0002:00001c38       ??_C@_0DO@FNIKKMPE@Couldn?8t?5find?5NativeGSSContext?$CI@ 0000000180008c38     NativeUtil.obj
 0002:00001c78       ??_C@_04OHLIFDMD@?$CIJ?$CJV@ 0000000180008c78     NativeUtil.obj
 0002:00001c80       ??_C@_0L@JADAHEAA@setContext@ 0000000180008c80     NativeUtil.obj
 0002:00001c90       ??_C@_0DI@LJLAMGFN@Couldn?8t?5find?5NativeGSSContext?4@ 0000000180008c90     NativeUtil.obj
 0002:00001cc8       ??_C@_0CF@GLMFJBKG@sun?1security?1jgss?1wrapper?1GSSLi@ 0000000180008cc8     NativeUtil.obj
 0002:00001cf0       ??_C@_0DK@DKLJHFGN@Couldn?8t?5find?5sun?4security?4jgss@ 0000000180008cf0     NativeUtil.obj
 0002:00001d2c       ??_C@_01LELAEKIP@J@        0000000180008d2c     NativeUtil.obj
 0002:00001d30       ??_C@_05ODBFMIC@pMech@     0000000180008d30     NativeUtil.obj
 0002:00001d38       ??_C@_0CG@KDHAILGJ@Couldn?8t?5find?5GSSLibStub?4pMech?5@ 0000000180008d38     NativeUtil.obj
 0002:00001d60       ??_C@_08BAFMHLII@pContext@ 0000000180008d60     NativeUtil.obj
 0002:00001d70       ??_C@_0CP@ENCPPLKK@Couldn?8t?5find?5NativeGSSContext?4@ 0000000180008d70     NativeUtil.obj
 0002:00001da0       ??_C@_0CL@POIDEFHJ@Lsun?1security?1jgss?1wrapper?1GSSN@ 0000000180008da0     NativeUtil.obj
 0002:00001dd0       ??_C@_07HBEJLLMM@srcName@  0000000180008dd0     NativeUtil.obj
 0002:00001dd8       ??_C@_0CO@DONIBCN@Couldn?8t?5find?5NativeGSSContext?4@ 0000000180008dd8     NativeUtil.obj
 0002:00001e08       ??_C@_0L@JFDMNPJH@targetName@ 0000000180008e08     NativeUtil.obj
 0002:00001e18       ??_C@_0DB@DDBEJNEH@Couldn?8t?5find?5NativeGSSContext?4@ 0000000180008e18     NativeUtil.obj
 0002:00001e4c       ??_C@_01POHCFINO@Z@        0000000180008e4c     NativeUtil.obj
 0002:00001e50       ??_C@_0M@EGOKMCMC@isInitiator@ 0000000180008e50     NativeUtil.obj
 0002:00001e60       ??_C@_0DC@LNCJDFLL@Couldn?8t?5find?5NativeGSSContext?4@ 0000000180008e60     NativeUtil.obj
 0002:00001e98       ??_C@_0O@IOAFJPFC@isEstablished@ 0000000180008e98     NativeUtil.obj
 0002:00001ea8       ??_C@_0DE@LNDCMEKK@Couldn?8t?5find?5NativeGSSContext?4@ 0000000180008ea8     NativeUtil.obj
 0002:00001ee0       ??_C@_0CL@JHCIJAHA@Lsun?1security?1jgss?1wrapper?1GSSC@ 0000000180008ee0     NativeUtil.obj
 0002:00001f10       ??_C@_0O@CPAICCNI@delegatedCred@ 0000000180008f10     NativeUtil.obj
 0002:00001f20       ??_C@_0DE@DKEHMLGM@Couldn?8t?5find?5NativeGSSContext?4@ 0000000180008f20     NativeUtil.obj
 0002:00001f54       ??_C@_01JPJNBJEM@I@        0000000180008f54     NativeUtil.obj
 0002:00001f58       ??_C@_05GECEPKB@flags@     0000000180008f58     NativeUtil.obj
 0002:00001f60       ??_C@_0CM@DLHPFAAC@Couldn?8t?5find?5NativeGSSContext?4@ 0000000180008f60     NativeUtil.obj
 0002:00001f90       ??_C@_08MOKDPMFA@lifetime@ 0000000180008f90     NativeUtil.obj
 0002:00001fa0       ??_C@_0CP@NKFJJLMO@Couldn?8t?5find?5NativeGSSContext?4@ 0000000180008fa0     NativeUtil.obj
 0002:00001fd0       ??_C@_0BE@LEBOECLA@Lorg?1ietf?1jgss?1Oid?$DL@ 0000000180008fd0     NativeUtil.obj
 0002:00001fe8       ??_C@_0L@GPNEDCNK@actualMech@ 0000000180008fe8     NativeUtil.obj
 0002:00001ff8       ??_C@_0DB@ENGNPLHP@Couldn?8t?5find?5NativeGSSContext?4@ 0000000180008ff8     NativeUtil.obj
 0002:00002030       ??_C@_0BL@ENCPOIKC@java?1lang?1OutOfMemoryError@ 0000000180009030     NativeUtil.obj
 0002:00002050       ??_C@_0CP@KLPLCPB@?$FLGSSLibStub?3?$CFd?$FN?5?$CFs?5Status?5major@ 0000000180009050     NativeUtil.obj
 0002:00002080       ??_C@_0CD@EABHFLMM@?$FLGSSLibStub?3?$CFd?$FN?5c?1r?1s?5?$DN?5?$CFd?1?$CFd?1?$CF@ 0000000180009080     NativeUtil.obj
 0002:000020a8       ??_C@_0CK@DNKNKJGD@A?5required?5input?5parameter?5cann@ 00000001800090a8     NativeUtil.obj
 0002:000020d8       ??_C@_0CM@BAFDHAPF@A?5required?5output?5parameter?5can@ 00000001800090d8     NativeUtil.obj
 0002:00002108       ??_C@_0BK@ONEELEFA@A?5parameter?5was?5malformed@ 0000000180009108     NativeUtil.obj
 0002:00002128       _pDefaultRawDllMain        0000000180009128     MSVCRT:dll_dllmain.obj
 0002:00002128       _pRawDllMain               0000000180009128     MSVCRT:dll_dllmain.obj
 0002:00002140       __xmm@ffffffffffffffffffffffffffffffff 0000000180009140     MSVCRT:utility.obj
 0002:00002150       _load_config_used          0000000180009150     MSVCRT:loadcfg.obj
 0002:00002300       __volatile_metadata        0000000180009300     <linker-defined>
 0002:00002628       __rtc_iaa                  0000000180009628     MSVCRT:initsect.obj
 0002:00002630       __rtc_izz                  0000000180009630     MSVCRT:initsect.obj
 0002:00002638       __rtc_taa                  0000000180009638     MSVCRT:initsect.obj
 0002:00002640       __rtc_tzz                  0000000180009640     MSVCRT:initsect.obj
 0002:00003208       __IMPORT_DESCRIPTOR_KERNEL32 000000018000a208     kernel32:KERNEL32.dll
 0002:0000321c       __IMPORT_DESCRIPTOR_VCRUNTIME140 000000018000a21c     vcruntime:VCRUNTIME140.dll
 0002:00003230       __IMPORT_DESCRIPTOR_api-ms-win-crt-stdio-l1-1-0 000000018000a230     ucrt:api-ms-win-crt-stdio-l1-1-0.dll
 0002:00003244       __IMPORT_DESCRIPTOR_api-ms-win-crt-heap-l1-1-0 000000018000a244     ucrt:api-ms-win-crt-heap-l1-1-0.dll
 0002:00003258       __IMPORT_DESCRIPTOR_api-ms-win-crt-runtime-l1-1-0 000000018000a258     ucrt:api-ms-win-crt-runtime-l1-1-0.dll
 0002:0000326c       __NULL_IMPORT_DESCRIPTOR   000000018000a26c     kernel32:KERNEL32.dll
 0003:00000000       __security_cookie          000000018000b000     MSVCRT:gs_cookie.obj
 0003:00000040       __security_cookie_complement 000000018000b040     MSVCRT:gs_cookie.obj
 0003:00000048       __scrt_native_dllmain_reason 000000018000b048     MSVCRT:utility.obj
 0003:00000050       __isa_inverted             000000018000b050     MSVCRT:cpu_disp.obj
 0003:00000058       __isa_available            000000018000b058     MSVCRT:cpu_disp.obj
 0003:0000005c       __isa_enabled              000000018000b05c     MSVCRT:cpu_disp.obj
 0003:00000060       __memset_fast_string_threshold 000000018000b060     MSVCRT:cpu_disp.obj
 0003:00000068       __memset_nt_threshold      000000018000b068     MSVCRT:cpu_disp.obj
 0003:00000070       __scrt_ucrt_dll_is_in_use  000000018000b070     MSVCRT:ucrt_stubs.obj
 0003:00000710       ?__type_info_root_node@@3U__type_info_node@@A 000000018000b710     MSVCRT:tncleanup.obj
 0003:00000720       ?_OptionsStorage@?1??__local_stdio_scanf_options@@9@4_KA 000000018000b720     MSVCRT:default_local_stdio_options.obj
 0003:00000728       __scrt_current_native_startup_state 000000018000b728     MSVCRT:utility.obj
 0003:00000730       __scrt_native_startup_lock 000000018000b730     MSVCRT:utility.obj
 0003:00000770       __scrt_debugger_hook_flag  000000018000b770     MSVCRT:utility_desktop.obj
 0003:00000774       __avx10_version            000000018000b774     MSVCRT:cpu_disp.obj
 0003:00000778       __favor                    000000018000b778     MSVCRT:cpu_disp.obj
 0003:00000780       MID_GSSException_ctor3     000000018000b780     <common>
 0003:00000788       MID_Oid_getDER             000000018000b788     <common>
 0003:00000790       MID_Oid_ctor1              000000018000b790     <common>
 0003:00000798       MID_String_ctor            000000018000b798     <common>
 0003:000007a0       CLS_SunNativeProvider      000000018000b7a0     <common>
 0003:000007a8       CLS_GSSException           000000018000b7a8     <common>
 0003:000007b0       CLS_Oid                    000000018000b7b0     <common>
 0003:000007b8       CLS_String                 000000018000b7b8     <common>
 0003:000007c0       FID_NativeGSSContext_actualMech 000000018000b7c0     <common>
 0003:000007c8       FID_NativeGSSContext_lifetime 000000018000b7c8     <common>
 0003:000007d0       FID_NativeGSSContext_flags 000000018000b7d0     <common>
 0003:000007d8       FID_NativeGSSContext_delegatedCred 000000018000b7d8     <common>
 0003:000007e0       FID_NativeGSSContext_isEstablished 000000018000b7e0     <common>
 0003:000007e8       FID_NativeGSSContext_isInitiator 000000018000b7e8     <common>
 0003:000007f0       FID_NativeGSSContext_targetName 000000018000b7f0     <common>
 0003:000007f8       FID_NativeGSSContext_srcName 000000018000b7f8     <common>
 0003:00000800       FID_NativeGSSContext_pContext 000000018000b800     <common>
 0003:00000808       FID_GSSLibStub_pMech       000000018000b808     <common>
 0003:00000810       MID_NativeGSSContext_setContext 000000018000b810     <common>
 0003:00000818       MID_NativeGSSContext_ctor  000000018000b818     <common>
 0003:00000820       MID_GSSCredElement_ctor    000000018000b820     <common>
 0003:00000828       MID_GSSNameElement_ctor    000000018000b828     <common>
 0003:00000830       MID_InetAddress_getAddr    000000018000b830     <common>
 0003:00000838       MID_ChannelBinding_getAppData 000000018000b838     <common>
 0003:00000840       MID_ChannelBinding_getAcceptorAddr 000000018000b840     <common>
 0003:00000848       MID_ChannelBinding_getInitiatorAddr 000000018000b848     <common>
 0003:00000850       MID_MessageProp_setSupplementaryStates 000000018000b850     <common>
 0003:00000858       MID_MessageProp_setQOP     000000018000b858     <common>
 0003:00000860       MID_MessageProp_setPrivacy 000000018000b860     <common>
 0003:00000868       MID_MessageProp_getQOP     000000018000b868     <common>
 0003:00000870       MID_MessageProp_getPrivacy 000000018000b870     <common>
 0003:00000878       CLS_NativeGSSContext       000000018000b878     <common>
 0003:00000880       CLS_GSSCredElement         000000018000b880     <common>
 0003:00000888       CLS_GSSNameElement         000000018000b888     <common>
 0003:00000890       CLS_Object                 000000018000b890     <common>
 0003:00000898       JGSS_DEBUG                 000000018000b898     <common>
 0003:000008a0       ftab                       000000018000b8a0     <common>
 0003:000008a8       ?_OptionsStorage@?1??__local_stdio_printf_options@@9@9 000000018000b8a8     <common>
 0003:000008b0       __dyn_tls_init_callback    000000018000b8b0     <common>

 entry point at        0001:00004d50

 Static symbols

 0000:ffff1000       .debug$S                   0000000180000000     j2gss.exp
 0000:ffff1000       .debug$S                   0000000180000000     vcruntime:VCRUNTIME140.dll
 0000:ffff1000       .debug$S                   0000000180000000     vcruntime:VCRUNTIME140.dll
 0000:ffff1000       .debug$S                   0000000180000000     vcruntime:VCRUNTIME140.dll
 0000:ffff1000       .debug$S                   0000000180000000     vcruntime:VCRUNTIME140.dll
 0000:ffff1000       .debug$S                   0000000180000000     vcruntime:VCRUNTIME140.dll
 0000:ffff1000       .debug$S                   0000000180000000     vcruntime:VCRUNTIME140.dll
 0000:ffff1000       .debug$S                   0000000180000000     vcruntime:VCRUNTIME140.dll
 0000:ffff1000       .debug$S                   0000000180000000     ucrt:api-ms-win-crt-heap-l1-1-0.dll
 0000:ffff1000       .debug$S                   0000000180000000     ucrt:api-ms-win-crt-heap-l1-1-0.dll
 0000:ffff1000       .debug$S                   0000000180000000     ucrt:api-ms-win-crt-heap-l1-1-0.dll
 0000:ffff1000       .debug$S                   0000000180000000     ucrt:api-ms-win-crt-runtime-l1-1-0.dll
 0000:ffff1000       .debug$S                   0000000180000000     ucrt:api-ms-win-crt-runtime-l1-1-0.dll
 0000:ffff1000       .debug$S                   0000000180000000     ucrt:api-ms-win-crt-runtime-l1-1-0.dll
 0000:ffff1000       .debug$S                   0000000180000000     ucrt:api-ms-win-crt-runtime-l1-1-0.dll
 0000:ffff1000       .debug$S                   0000000180000000     ucrt:api-ms-win-crt-runtime-l1-1-0.dll
 0000:ffff1000       .debug$S                   0000000180000000     ucrt:api-ms-win-crt-runtime-l1-1-0.dll
 0000:ffff1000       .debug$S                   0000000180000000     ucrt:api-ms-win-crt-runtime-l1-1-0.dll
 0000:ffff1000       .debug$S                   0000000180000000     ucrt:api-ms-win-crt-runtime-l1-1-0.dll
 0000:ffff1000       .debug$S                   0000000180000000     ucrt:api-ms-win-crt-runtime-l1-1-0.dll
 0000:ffff1000       .debug$S                   0000000180000000     ucrt:api-ms-win-crt-runtime-l1-1-0.dll
 0000:ffff1000       .debug$S                   0000000180000000     ucrt:api-ms-win-crt-runtime-l1-1-0.dll
 0000:ffff1000       .debug$S                   0000000180000000     ucrt:api-ms-win-crt-runtime-l1-1-0.dll
 0000:ffff1000       .debug$S                   0000000180000000     ucrt:api-ms-win-crt-stdio-l1-1-0.dll
 0000:ffff1000       .debug$S                   0000000180000000     ucrt:api-ms-win-crt-stdio-l1-1-0.dll
 0000:ffff1000       .debug$S                   0000000180000000     ucrt:api-ms-win-crt-stdio-l1-1-0.dll
 0000:ffff1000       .debug$S                   0000000180000000     kernel32:KERNEL32.dll
 0000:ffff1000       .debug$S                   0000000180000000     kernel32:KERNEL32.dll
 0000:ffff1000       .debug$S                   0000000180000000     kernel32:KERNEL32.dll
 0000:ffff1000       .debug$S                   0000000180000000     kernel32:KERNEL32.dll
 0000:ffff1000       .debug$S                   0000000180000000     kernel32:KERNEL32.dll
 0000:ffff1000       .debug$S                   0000000180000000     kernel32:KERNEL32.dll
 0000:ffff1000       .debug$S                   0000000180000000     kernel32:KERNEL32.dll
 0000:ffff1000       .debug$S                   0000000180000000     kernel32:KERNEL32.dll
 0000:ffff1000       .debug$S                   0000000180000000     kernel32:KERNEL32.dll
 0000:ffff1000       .debug$S                   0000000180000000     kernel32:KERNEL32.dll
 0000:ffff1000       .debug$S                   0000000180000000     kernel32:KERNEL32.dll
 0000:ffff1000       .debug$S                   0000000180000000     kernel32:KERNEL32.dll
 0000:ffff1000       .debug$S                   0000000180000000     kernel32:KERNEL32.dll
 0000:ffff1000       .debug$S                   0000000180000000     kernel32:KERNEL32.dll
 0000:ffff1000       .debug$S                   0000000180000000     kernel32:KERNEL32.dll
 0000:ffff1000       .debug$S                   0000000180000000     kernel32:KERNEL32.dll
 0000:ffff1000       .debug$S                   0000000180000000     kernel32:KERNEL32.dll
 0000:ffff1000       .debug$S                   0000000180000000     kernel32:KERNEL32.dll
 0000:ffff1000       .debug$S                   0000000180000000     kernel32:KERNEL32.dll
 0000:ffff1000       .debug$S                   0000000180000000     kernel32:KERNEL32.dll
 0000:ffff1000       .debug$S                   0000000180000000     kernel32:KERNEL32.dll
 0000:ffff1000       .debug$S                   0000000180000000     kernel32:KERNEL32.dll
 0001:00004a10       $$000000                   0000000180005a10     MSVCRT:amdsecgs.obj
 0001:00004a40       ?dllmain_crt_dispatch@@YAHQEAUHINSTANCE__@@KQEAX@Z 0000000180005a40 f   MSVCRT:dll_dllmain.obj
 0001:00004a90       ?dllmain_crt_process_attach@@YAHQEAUHINSTANCE__@@QEAX@Z 0000000180005a90 f   MSVCRT:dll_dllmain.obj
 0001:00004ba8       ?dllmain_crt_process_detach@@YAH_N@Z 0000000180005ba8 f   MSVCRT:dll_dllmain.obj
 0001:00004c28       ?dllmain_dispatch@@YAHQEAUHINSTANCE__@@KQEAX@Z 0000000180005c28 f   MSVCRT:dll_dllmain.obj
 0001:00004e98       capture_previous_context   0000000180005e98 f   MSVCRT:gs_report.obj
 0001:00005850       $$000000                   0000000180006850     MSVCRT:guard_dispatch.obj
 0001:00005870       $$000000                   0000000180006870     MSVCRT:guard_xfg_dispatch.obj
 0001:00005886       ?fin$0@?0??dllmain_crt_process_attach@@YAHQEAUHINSTANCE__@@QEAX@Z@4HA 0000000180006886 f   MSVCRT:dll_dllmain.obj
 0001:0000589d       ?fin$0@?0??dllmain_crt_process_detach@@YAH_N@Z@4HA 000000018000689d f   MSVCRT:dll_dllmain.obj
 0001:000058b6       ?fin$1@?0??dllmain_crt_process_detach@@YAH_N@Z@4HA 00000001800068b6 f   MSVCRT:dll_dllmain.obj
 0001:000058ca       ?filt$0@?0??dllmain_dispatch@@YAHQEAUHINSTANCE__@@KQEAX@Z@4HA 00000001800068ca f   MSVCRT:dll_dllmain.obj
 0001:00005900       __scrt_is_nonwritable_in_current_image$filt$0 0000000180006900 f   MSVCRT:utility.obj
 0002:00001098       RELEASE_NAME               0000000180008098     NativeFunc.obj
 0002:000010b0       IMPORT_NAME                00000001800080b0     NativeFunc.obj
 0002:000010c0       COMPARE_NAME               00000001800080c0     NativeFunc.obj
 0002:000010d8       CANONICALIZE_NAME          00000001800080d8     NativeFunc.obj
 0002:000010f0       EXPORT_NAME                00000001800080f0     NativeFunc.obj
 0002:00001100       DISPLAY_NAME               0000000180008100     NativeFunc.obj
 0002:00001118       ACQUIRE_CRED               0000000180008118     NativeFunc.obj
 0002:00001130       RELEASE_CRED               0000000180008130     NativeFunc.obj
 0002:00001148       INQUIRE_CRED               0000000180008148     NativeFunc.obj
 0002:00001160       IMPORT_SEC_CONTEXT         0000000180008160     NativeFunc.obj
 0002:00001178       INIT_SEC_CONTEXT           0000000180008178     NativeFunc.obj
 0002:00001190       ACCEPT_SEC_CONTEXT         0000000180008190     NativeFunc.obj
 0002:000011a8       INQUIRE_CONTEXT            00000001800081a8     NativeFunc.obj
 0002:000011c0       DELETE_SEC_CONTEXT         00000001800081c0     NativeFunc.obj
 0002:000011d8       CONTEXT_TIME               00000001800081d8     NativeFunc.obj
 0002:000011f0       WRAP_SIZE_LIMIT            00000001800081f0     NativeFunc.obj
 0002:00001208       EXPORT_SEC_CONTEXT         0000000180008208     NativeFunc.obj
 0002:00001220       GET_MIC                    0000000180008220     NativeFunc.obj
 0002:00001230       VERIFY_MIC                 0000000180008230     NativeFunc.obj
 0002:00001240       WRAP                       0000000180008240     NativeFunc.obj
 0002:00001250       UNWRAP                     0000000180008250     NativeFunc.obj
 0002:00001260       INDICATE_MECHS             0000000180008260     NativeFunc.obj
 0002:00001278       INQUIRE_NAMES_FOR_MECH     0000000180008278     NativeFunc.obj
 0002:00001298       ADD_OID_SET_MEMBER         0000000180008298     NativeFunc.obj
 0002:000012b0       DISPLAY_STATUS             00000001800082b0     NativeFunc.obj
 0002:000012c8       CREATE_EMPTY_OID_SET       00000001800082c8     NativeFunc.obj
 0002:000012e8       RELEASE_OID_SET            00000001800082e8     NativeFunc.obj
 0002:00001300       RELEASE_BUFFER             0000000180008300     NativeFunc.obj
 0002:00002130       GS_ExceptionPointers       0000000180009130     MSVCRT:gs_report.obj
 0002:00002648       $unwind$fprintf            0000000180009648     GSSLibStub.obj
 0002:00002654       $unwind$Java_sun_security_jgss_wrapper_GSSLibStub_init 0000000180009654     GSSLibStub.obj
 0002:0000266c       $unwind$Java_sun_security_jgss_wrapper_GSSLibStub_getMechPtr 000000018000966c     GSSLibStub.obj
 0002:00002684       $unwind$Java_sun_security_jgss_wrapper_GSSLibStub_compareName 0000000180009684     GSSLibStub.obj
 0002:00002684       $unwind$Java_sun_security_jgss_wrapper_GSSLibStub_inquireNamesForMech 0000000180009684     GSSLibStub.obj
 0002:00002694       $unwind$Java_sun_security_jgss_wrapper_GSSLibStub_canonicalizeName 0000000180009694     GSSLibStub.obj
 0002:00002694       $unwind$Java_sun_security_jgss_wrapper_GSSLibStub_deleteContext 0000000180009694     GSSLibStub.obj
 0002:00002694       $unwind$Java_sun_security_jgss_wrapper_GSSLibStub_getContextTime 0000000180009694     GSSLibStub.obj
 0002:00002694       $unwind$Java_sun_security_jgss_wrapper_GSSLibStub_releaseCred 0000000180009694     GSSLibStub.obj
 0002:00002694       $unwind$Java_sun_security_jgss_wrapper_GSSLibStub_releaseName 0000000180009694     GSSLibStub.obj
 0002:00002694       $unwind$newGSSOID          0000000180009694     NativeUtil.obj
 0002:000026a4       $unwind$Java_sun_security_jgss_wrapper_GSSLibStub_importName 00000001800096a4     GSSLibStub.obj
 0002:000026b8       $unwind$Java_sun_security_jgss_wrapper_GSSLibStub_displayName 00000001800096b8     GSSLibStub.obj
 0002:000026b8       $unwind$Java_sun_security_jgss_wrapper_GSSLibStub_exportContext 00000001800096b8     GSSLibStub.obj
 0002:000026b8       $unwind$Java_sun_security_jgss_wrapper_GSSLibStub_exportName 00000001800096b8     GSSLibStub.obj
 0002:000026cc       $unwind$Java_sun_security_jgss_wrapper_GSSLibStub_acquireCred 00000001800096cc     GSSLibStub.obj
 0002:000026e4       $unwind$Java_sun_security_jgss_wrapper_GSSLibStub_getCredName 00000001800096e4     GSSLibStub.obj
 0002:000026e4       $unwind$Java_sun_security_jgss_wrapper_GSSLibStub_getCredTime 00000001800096e4     GSSLibStub.obj
 0002:000026e4       $unwind$Java_sun_security_jgss_wrapper_GSSLibStub_getCredUsage 00000001800096e4     GSSLibStub.obj
 0002:000026f4       $unwind$Java_sun_security_jgss_wrapper_GSSLibStub_importContext 00000001800096f4     GSSLibStub.obj
 0002:00002708       $unwind$Java_sun_security_jgss_wrapper_GSSLibStub_initContext 0000000180009708     GSSLibStub.obj
 0002:00002724       $unwind$Java_sun_security_jgss_wrapper_GSSLibStub_acceptContext 0000000180009724     GSSLibStub.obj
 0002:00002740       $unwind$Java_sun_security_jgss_wrapper_GSSLibStub_inquireContext 0000000180009740     GSSLibStub.obj
 0002:0000275c       $unwind$Java_sun_security_jgss_wrapper_GSSLibStub_getContextMech 000000018000975c     GSSLibStub.obj
 0002:0000276c       $unwind$Java_sun_security_jgss_wrapper_GSSLibStub_getContextName 000000018000976c     GSSLibStub.obj
 0002:00002780       $unwind$Java_sun_security_jgss_wrapper_GSSLibStub_wrapSizeLimit 0000000180009780     GSSLibStub.obj
 0002:00002794       $unwind$Java_sun_security_jgss_wrapper_GSSLibStub_getMic 0000000180009794     GSSLibStub.obj
 0002:000027a8       $unwind$Java_sun_security_jgss_wrapper_GSSLibStub_verifyMic 00000001800097a8     GSSLibStub.obj
 0002:000027bc       $unwind$Java_sun_security_jgss_wrapper_GSSLibStub_wrap 00000001800097bc     GSSLibStub.obj
 0002:000027d4       $unwind$Java_sun_security_jgss_wrapper_GSSLibStub_unwrap 00000001800097d4     GSSLibStub.obj
 0002:000027ec       $unwind$deleteGSSCB        00000001800097ec     GSSLibStub.obj
 0002:000027ec       $unwind$deleteGSSOID       00000001800097ec     NativeUtil.obj
 0002:000027ec       $unwind$resetGSSBuffer     00000001800097ec     NativeUtil.obj
 0002:000027f4       $unwind$newGSSCB           00000001800097f4     GSSLibStub.obj
 0002:000027f4       $unwind$__scrt_dllmain_exception_filter 00000001800097f4     MSVCRT:utility.obj
 0002:00002808       $unwind$setSupplementaryInfo 0000000180009808     GSSLibStub.obj
 0002:00002820       $unwind$inquireCred        0000000180009820     GSSLibStub.obj
 0002:00002834       $unwind$loadNative         0000000180009834     NativeFunc.obj
 0002:00002834       $unwind$gssThrowOutOfMemoryError 0000000180009834     NativeUtil.obj
 0002:00002834       $unwind$_RTC_Initialize    0000000180009834     MSVCRT:initsect.obj
 0002:00002834       $unwind$_RTC_Terminate     0000000180009834     MSVCRT:initsect.obj
 0002:00002840       $unwind$JNI_OnLoad         0000000180009840     NativeUtil.obj
 0002:00002850       $unwind$JNI_OnUnload       0000000180009850     NativeUtil.obj
 0002:00002850       $unwind$__scrt_initialize_default_local_stdio_options 0000000180009850     MSVCRT:default_local_stdio_options.obj
 0002:00002850       $unwind$?dllmain_crt_dispatch@@YAHQEAUHINSTANCE__@@KQEAX@Z 0000000180009850     MSVCRT:dll_dllmain.obj
 0002:00002850       $unwind$DllMain            0000000180009850     MSVCRT:dll_dllmain_stub.obj
 0002:00002850       $unwind$__GSHandlerCheck   0000000180009850     MSVCRT:gshandler.obj
 0002:00002850       $unwind$__scrt_acquire_startup_lock 0000000180009850     MSVCRT:utility.obj
 0002:00002850       $unwind$__scrt_dllmain_after_initialize_c 0000000180009850     MSVCRT:utility.obj
 0002:00002850       $unwind$__scrt_dllmain_before_initialize_c 0000000180009850     MSVCRT:utility.obj
 0002:00002850       $unwind$__scrt_dllmain_crt_thread_attach 0000000180009850     MSVCRT:utility.obj
 0002:00002850       $unwind$__scrt_dllmain_crt_thread_detach 0000000180009850     MSVCRT:utility.obj
 0002:00002850       $unwind$__scrt_dllmain_uninitialize_c 0000000180009850     MSVCRT:utility.obj
 0002:00002850       $unwind$__scrt_dllmain_uninitialize_critical 0000000180009850     MSVCRT:utility.obj
 0002:00002850       $unwind$__scrt_initialize_crt 0000000180009850     MSVCRT:utility.obj
 0002:00002858       $unwind$checkStatus        0000000180009858     NativeUtil.obj
 0002:00002874       $unwind$initGSSBuffer      0000000180009874     NativeUtil.obj
 0002:0000288c       $unwind$newGSSOIDSet       000000018000988c     NativeUtil.obj
 0002:0000288c       $unwind$sameMech           000000018000988c     NativeUtil.obj
 0002:0000288c       $unwind$__raise_securityfailure 000000018000988c     MSVCRT:gs_report.obj
 0002:0000288c       $unwind$__scrt_initialize_onexit_tables 000000018000988c     MSVCRT:utility.obj
 0002:0000288c       $unwind$__scrt_release_startup_lock 000000018000988c     MSVCRT:utility.obj
 0002:0000288c       $unwind$__scrt_uninitialize_crt 000000018000988c     MSVCRT:utility.obj
 0002:00002894       $unwind$deleteGSSOIDSet    0000000180009894     NativeUtil.obj
 0002:0000289c       $unwind$getJavaBuffer      000000018000989c     NativeUtil.obj
 0002:000028b0       $unwind$getJavaString      00000001800098b0     NativeUtil.obj
 0002:000028c4       $unwind$getJavaOID         00000001800098c4     NativeUtil.obj
 0002:000028d8       $unwind$getJavaOIDArray    00000001800098d8     NativeUtil.obj
 0002:000028f0       $unwind$getMinorMessage    00000001800098f0     NativeUtil.obj
 0002:000028fc       $unwind$__GSHandlerCheckCommon 00000001800098fc     MSVCRT:gshandler.obj
 0002:00002908       $xdatasym                  0000000180009908     MSVCRT:amdsecgs.obj
 0002:0000290c       $unwind$?dllmain_crt_process_attach@@YAHQEAUHINSTANCE__@@QEAX@Z 000000018000990c     MSVCRT:dll_dllmain.obj
 0002:00002948       $unwind$?fin$0@?0??dllmain_crt_process_attach@@YAHQEAUHINSTANCE__@@QEAX@Z@4HA 0000000180009948     MSVCRT:dll_dllmain.obj
 0002:00002948       $unwind$?fin$0@?0??dllmain_crt_process_detach@@YAH_N@Z@4HA 0000000180009948     MSVCRT:dll_dllmain.obj
 0002:00002948       $unwind$?fin$1@?0??dllmain_crt_process_detach@@YAH_N@Z@4HA 0000000180009948     MSVCRT:dll_dllmain.obj
 0002:00002950       $unwind$?dllmain_crt_process_detach@@YAH_N@Z 0000000180009950     MSVCRT:dll_dllmain.obj
 0002:000029a4       $unwind$?dllmain_dispatch@@YAHQEAUHINSTANCE__@@KQEAX@Z 00000001800099a4     MSVCRT:dll_dllmain.obj
 0002:000029cc       $unwind$?filt$0@?0??dllmain_dispatch@@YAHQEAUHINSTANCE__@@KQEAX@Z@4HA 00000001800099cc     MSVCRT:dll_dllmain.obj
 0002:000029d4       $unwind$_DllMainCRTStartup 00000001800099d4     MSVCRT:dll_dllmain.obj
 0002:000029e4       $unwind$__report_gsfailure 00000001800099e4     MSVCRT:gs_report.obj
 0002:000029ec       $unwind$capture_previous_context 00000001800099ec     MSVCRT:gs_report.obj
 0002:000029f8       $unwind$__security_init_cookie 00000001800099f8     MSVCRT:gs_support.obj
 0002:00002a04       $unwind$__scrt_is_nonwritable_in_current_image 0000000180009a04     MSVCRT:utility.obj
 0002:00002a24       $unwind$__scrt_is_nonwritable_in_current_image$filt$0 0000000180009a24     MSVCRT:utility.obj
 0002:00002a2c       $unwind$__scrt_fastfail    0000000180009a2c     MSVCRT:utility_desktop.obj
 0002:00002a3c       $unwind$__isa_available_init 0000000180009a3c     MSVCRT:cpu_disp.obj
 0002:00002a50       $xdatasym                  0000000180009a50     MSVCRT:guard_dispatch.obj
 0002:00002a58       $xdatasym                  0000000180009a58     MSVCRT:guard_xfg_dispatch.obj
 0002:00002a60       .edata                     0000000180009a60     j2gss.exp
 0002:00002a88       rgpv                       0000000180009a88     j2gss.exp
 0002:00002b04       rgszName                   0000000180009b04     j2gss.exp
 0002:00002b80       rgwOrd                     0000000180009b80     j2gss.exp
 0002:00002bbe       szName                     0000000180009bbe     j2gss.exp
 0002:00002bc8       $N00001                    0000000180009bc8     j2gss.exp
 0002:00002bd3       $N00002                    0000000180009bd3     j2gss.exp
 0002:00002be0       $N00003                    0000000180009be0     j2gss.exp
 0002:00002c18       $N00004                    0000000180009c18     j2gss.exp
 0002:00002c4e       $N00005                    0000000180009c4e     j2gss.exp
 0002:00002c89       $N00006                    0000000180009c89     j2gss.exp
 0002:00002cbf       $N00007                    0000000180009cbf     j2gss.exp
 0002:00002cf7       $N00008                    0000000180009cf7     j2gss.exp
 0002:00002d2d       $N00009                    0000000180009d2d     j2gss.exp
 0002:00002d65       $N00010                    0000000180009d65     j2gss.exp
 0002:00002d9a       $N00011                    0000000180009d9a     j2gss.exp
 0002:00002dd3       $N00012                    0000000180009dd3     j2gss.exp
 0002:00002e0c       $N00013                    0000000180009e0c     j2gss.exp
 0002:00002e45       $N00014                    0000000180009e45     j2gss.exp
 0002:00002e7b       $N00015                    0000000180009e7b     j2gss.exp
 0002:00002eb1       $N00016                    0000000180009eb1     j2gss.exp
 0002:00002ee8       $N00017                    0000000180009ee8     j2gss.exp
 0002:00002f1d       $N00018                    0000000180009f1d     j2gss.exp
 0002:00002f4e       $N00019                    0000000180009f4e     j2gss.exp
 0002:00002f86       $N00020                    0000000180009f86     j2gss.exp
 0002:00002fbb       $N00021                    0000000180009fbb     j2gss.exp
 0002:00002ff3       $N00022                    0000000180009ff3     j2gss.exp
 0002:00003022       $N00023                    000000018000a022     j2gss.exp
 0002:00003058       $N00024                    000000018000a058     j2gss.exp
 0002:00003091       $N00025                    000000018000a091     j2gss.exp
 0002:000030cf       $N00026                    000000018000a0cf     j2gss.exp
 0002:00003105       $N00027                    000000018000a105     j2gss.exp
 0002:0000313b       $N00028                    000000018000a13b     j2gss.exp
 0002:0000316c       $N00029                    000000018000a16c     j2gss.exp
 0002:000031a0       $N00030                    000000018000a1a0     j2gss.exp
 0002:000031cf       $N00031                    000000018000a1cf     j2gss.exp
 0002:00003598       .idata$6                   000000018000a598     kernel32:KERNEL32.dll
 0002:000035f2       .idata$6                   000000018000a5f2     vcruntime:VCRUNTIME140.dll
 0002:000036fc       .idata$6                   000000018000a6fc     ucrt:api-ms-win-crt-stdio-l1-1-0.dll
 0002:0000371c       .idata$6                   000000018000a71c     ucrt:api-ms-win-crt-heap-l1-1-0.dll
 0002:0000373c       .idata$6                   000000018000a73c     ucrt:api-ms-win-crt-runtime-l1-1-0.dll
 0003:00000080       tlsCBCl                    000000018000b080     GSSLibStub.obj
 0003:00000090       ?szMsgBuf@?P@??Java_sun_security_jgss_wrapper_GSSLibStub_init@@9@9 000000018000b090     GSSLibStub.obj
 0003:00000190       ?__proc_attached@@3HA      000000018000b190     MSVCRT:dll_dllmain.obj
 0003:000001a0       GS_ExceptionRecord         000000018000b1a0     MSVCRT:gs_report.obj
 0003:00000240       GS_ContextRecord           000000018000b240     MSVCRT:gs_report.obj
 0003:00000738       ?is_initialized_as_dll@@3_NA 000000018000b738     MSVCRT:utility.obj
 0003:00000739       ?module_local_atexit_table_initialized@@3_NA 000000018000b739     MSVCRT:utility.obj
 0003:00000740       ?module_local_atexit_table@@3U_onexit_table_t@@A 000000018000b740     MSVCRT:utility.obj
 0003:00000758       ?module_local_at_quick_exit_table@@3U_onexit_table_t@@A 000000018000b758     MSVCRT:utility.obj
 0005:00000060       $R000000                   000000018000d060     j2gss.dll.res
